:1000000006C1000016C1000014C1000012C10000AA
:1000100010C100000EC100000CC100000AC10000A8
:1000200008C1000006C1000004C1000002C10000B8
:1000300000C10000FEC00000FCC00000FAC00000CB
:10004000F8C00000F6C00000F4C00000F2C00000DC
:10005000F0C00000EEC00000ECC00000EBC00000EB
:10006000E8C00000E6C00000E4C00000E2C00000FC
:10007000E0C00000DEC00000DCC00000DAC000000C
:10008000D8C00000D6C00000D4C00000D2C000001C
:10009000D0C00000CEC00000CCC00000CAC000002C
:1000A000C8C00000C6C00000C4C00000C2C000003C
:1000B000C0C00000BEC00000BCC00000BAC000004C
:1000C000B8C00000B6C00000B4C00000B2C000005C
:1000D000B0C00000AEC00000ACC00000AAC000006C
:1000E000A8C000002402270216021A021E025E02A5
:1000F0002B022F02350239023D02430247024B0216
:100100005E0251025502590200002100240027001E
:100110002A002D0030003300010100000401070116
:100120000A0100002200250028002B002E003100CB
:10013000340002010000050108010B010505050559
:10014000070508080808020202020A0A080804044F
:10015000040401010101010101010303030303037D
:100160000303040707070C0C0C0C0C0C0C0C02020C
:10017000020206060606060606060B0B0B0B0B0B09
:100180000B0B010210202008081020401020408096
:10019000020102010804020101020408102040804B
:1001A00080402010080402018004020180402010D9
:1001B0000804020108040201010204081020408022
:1001C000010204081020408000000A0B02090C0DF7
:1001D0000E080703040100000000000000000000FA
:1001E000000000000000000000000000000000000F
:1001F00000000000121110000000000000000000CC
:1002000000000000000000000000000000001124B9
:100210001FBECFEFD1E2DEBFCDBF00E00CBF22E0BA
:10022000A0E0B2E001C01D92A930B207E1F74CD0C6
:1002300070C1E6CE1F920F920FB60F9211242F932A
:100240003F938F939F93AF93BF93809105029091BB
:100250000602A0910702B09108023091040223E047
:10026000230F2D3720F40196A11DB11D05C026E8EE
:10027000230F0296A11DB11D209304028093050255
:1002800090930602A0930702B093080280910002A7
:1002900090910102A0910202B09103020196A11D6A
:1002A000B11D8093000290930102A0930202B093CB
:1002B0000302BF91AF919F918F913F912F910F902A
:1002C0000FBE0F901F901895789484B5826084BDFE
:1002D00084B5816084BD85B5826085BD85B581604A
:1002E00085BD80916E00816080936E0010928100C8
:1002F0008091810082608093810080918100816083
:100300008093810080918000816080938000809143
:10031000B10084608093B1008091B00081608093CF
:10032000B000809191008260809391008091910053
:100330008160809391008091900081608093900013
:100340008091A10082608093A1008091A1008160D2
:100350008093A1008091A00081608093A000809193
:10036000210182608093210180912101816080932D
:1003700021018091200181608093200180917A0089
:10038000846080937A0080917A00826080937A0002
:1003900080917A00816080937A0080917A008068F1
:1003A00080937A001092C1000FE811E0F8012491C7
:1003B000C9E4D1E0FE018491882399F090E0880F90
:1003C000991FFC01E85FFE4FA591B4918E5D9E4F91
:1003D000FC01459154918FB7F8949C91292B2C9353
:1003E0008FBFE12CF12C60E0C70185D0FFEFEF1A41
:1003F000FF0AE11480E1F806B1F7E5EDF1E0849140
:10040000F8010491FE01C491CC2309F465C088234E
:1004100009F454C090E0FC013197E231F10508F095
:100420004DC08827EE58FF4F8F4F5DC080918000F0
:100430008F7707C0809180008F7D03C080918000FE
:10044000877F809380003AC084B58F7702C084B5DF
:100450008F7D84BD33C08091B0008F7703C08091C1
:10046000B0008F7D8093B00029C0809190008F777D
:1004700007C0809190008F7D03C080919000877F9E
:10048000809390001BC08091A0008F7707C080915F
:10049000A0008F7D03C08091A000877F8093A00083
:1004A0000DC0809120018F7707C0809120018F7D42
:1004B00003C080912001877F80932001EC2FF0E022
:1004C000EE0FFF1FEE5DFE4FA591B4918FB7F8942C
:1004D0009C91092B0C938FBFC0E0D0E02097F1F3E3
:1004E0000E940000FBCFEE0FFF1F881F8BBF0790FD
:1004F000F691E02D1994262FF999FECF1FBA92BDDF
:1005000081BD20BD0FB6F894FA9AF99A0FBE0196F4
:060510000895F894FFCFEE
:00000001FF
